:1000000059C068C372C071C070C06FC06EC06DC08F
:100010006CC06BC06AC069C068C067C066C00501BB
:100020000906A101050719E029E715002501750159
:1000300095088102950175082565190029658100DB
:10004000C004030904240369006D0061006B0065AE
:1000500000700072006F006A006500630074007336
:10006000002E0063006F006D0016034800610075EC
:10007000006E0074006500640055005300420012D9
:1000800001100100000008424231E10001010200BC
:100090000109022200010100801909040000010386
:1000A000000000092101010001222300070581034E
:1000B00008000A0011241FBECFE5D1E0DEBFCDBF8E
:1000C00010E0A0E6B0E0EAE8FBE002C005900D9287
:1000D000A836B107D9F710E0A8E6B0E001C01D923C
:1000E000A83AB107E1F7B0D04FC58ACFEF92FF929F
:1000F0000F931F937B018C01FFE0EE0CFF1C001F90
:10010000111FFA95D1F72FEF3FEF4FEF5FE7E22294
:10011000F322042315239B01AC01E5E15595479596
:1001200037952795EA95D1F7E21AF30A040B150BD8
:100130009C01552737FD5095452FE20EF31E041FF5
:10014000151F2AE0660F771F881F991F2A95D1F780
:100150009F77E61AF70A080B190B17FF08C08FEFF5
:100160009FEFAFEFBFE7E80EF91E0A1F1B1FC80184
:10017000B7011F910F91FF90EF90089555D4AA27D2
:1001800097FDA095BA2FBC01CD01B0DF672F70E0BD
:1001900080E090E020E230E040E050E054D42115CF
:1001A00031054105510509F443C0213031054105B0
:1001B000510511F499E414C022303105410551056F
:1001C00011F49AE214C0233031054105510591F133
:1001D000243031054105510511F493E515C090E037
:1001E000253031054105510511F49BE20DC0263043
:1001F00031054105510511F49CE406C02730310555
:100200004105510509F499E320916D00222311F075
:1002100080E012C080917000882341F0833011F09B
:1002200099E301C090E0815080937000892F04C051
:1002300099E3D6CF9CE2E8CF2F5F20936D00109218
:100240006A0080936B000895CF93DF93A0E0B0E045
:1002500037D4802D8F3F09F081BFB89A20E083EB1F
:1002600091EF0197F1F72F5F2431C9F7B89888E132
:1002700090E02EE00FB6F894A89581BD0FBE21BD89
:100280008BE080BF88EC90E090936F0080936E00CD
:1002900083E080937000ABD07894CAE6D0E0A89554
:1002A000D2D08091620084FF08C080916D008230BE
:1002B00020F464DF62E0CE01A4D008B602FEEFCFE6
:1002C00084E088BF809168009091690001969093C6
:1002D00069008093680020916E0030916F00821752
:1002E0009307E8F2A1D38D5E944F90936F008093B3
:1002F0006E0080917000823030F08CE390E090933B
:100300006F0080936E001092690010926800109246
:100310006D00C5CFFC018AE690E090938D0080933C
:100320008C00808180768032D1F48181813021F40B
:1003300025DF82E090E00895823049F48CE690E079
:1003400090938D0080938C0081E090E008958A3036
:1003500031F4838180936C0080E090E0089580E028
:1003600090E00895DF92EF92FF920F931F93CF9347
:10037000DF93A0E8DA2EFF24C0E0D0E0EF2CED0CF4
:10038000E1BE95D18C0189E0043318070CF4FE2CF2
:10039000D6942196C830D10589F7FA94F1BEF3942A
:1003A000CF2DD0E0219610C082D18453994097FF81
:1003B00003C0909581959F4F8017910714F4F1B673
:1003C0008C0181B78F5F81BF81B790E0C817D907D3
:1003D0005CF7F1BE81B7A0E0B0E0082E79D3DF91E1
:1003E000CF911F910F91FF90EF90DF90089585B707
:1003F000836085BF8BB780648BBF83EC80937E0066
:1004000008951F93DC01162F8091620084FF07C0BE
:1004100080917E0098E8892780937E0003C08AE55A
:1004200080936200912FEFE7F0E002C08D918193FD
:100430009150E0F7612F8FE790E035D11C5F10936A
:1004400062001F9108950F931F93CF93DF939091B4
:100450008E0019160CF0ADC020918B0080918A009F
:100460008D3209F09EC08AE5809361009B3009F0CF
:1004700098C0CEE9D0E0C21BD1098881807609F00E
:1004800081C02CE730E010927C008981882341F400
:1004900010927D0030938D0020938C0092E075C007
:1004A000853021F48A8180938F006AC0863009F0FC
:1004B0004BC08B81813041F48FE790E090938D00A9
:1004C00080938C0092E164C0823041F481E990E035
:1004D00090938D0080938C0092E25AC0833001F596
:1004E0008A81882341F481E490E090938D00809389
:1004F0008C0094E04DC0813041F485E490E090930D
:100500008D0080938C0094E243C0823009F03FC09C
:1005100089E690E090938D0080938C0096E138C03E
:10052000813241F483EA90E090938D0080938C00B7
:1005300099E02EC0823259F58EE190E090938D00C3
:1005400080938C0093E224C0883039F481E990E0F4
:1005500090938D0080938C000CC0893021F48A81A7
:10056000809391000DC08A3031F430938D00209338
:100570008C0091E00AC08B3019F483EC80937E00EC
:1005800090E003C0CE01C6DE982F20E802C090E0C4
:1005900020EC8F81882339F48E81891720F4982FDD
:1005A00002C090E020E820937200909360001092C7
:1005B0008E008091610084FF45C0809160008F3F74
:1005C00009F440C0182F893008F018E0811B80938F
:1005D00060008091720080FF02C003EC01C00BE458
:1005E0008F5F8093720020918C0030918D0086FD8A
:1005F00005C0912FF901A4E7B0E00DC0912FF901DA
:10060000A4E7B0E003C084918D9331969150D8F760
:1006100004C081918D939150E0F7C901810F911D24
:1006200090938D0080938C00612F84E790E03BD005
:10063000183019F08FEF80936000009373001C5FF7
:10064000109361009AE086B3857031F49150D9F728
:1006500010928F001092890010E0992309F411E0A4
:1006600080917100811729F0112309F47BDE10932A
:100670007100DF91CF911F910F910895A82FB92F8D
:1006800080E090E041E050EA60956F5F58F42D9172
:1006900038EF82279795879510F0842795273F5F3D
:1006A000C8F3F3CF0895EADF8D939D930895A6E0F4
:1006B00088279927AA9569F00197E1F3B099FCCFB3
:1006C000B09BFECF81E09927A6B3019611F0A570EB
:1006D000D9F70895CF93CFB7CF93B09BFECFB09B00
:1006E0000BC0B09B09C0B09B07C0B09B05C0B09BBE
:1006F00003C0B09B01C0D5C00F92DF93C0918B00A7
:10070000DD27CE56DF4F012EB09B03C0DF910F9047
:10071000E6CF2F930F931F934F932FEF4F6F06B397
:1007200000FB20F95F933F9350E03BE065C016B3B8
:100730000126502950FDC89556B3012700FB25F925
:100740002F7306B3B1F05027102710FB26F906B21D
:100750002230F0F000C016B3012700FB27F9012674
:10076000502906B22430E8F54F77206816B3000010
:10077000F6CF50274F7D206206B2102F000000C038
:1007800006B300265029102710FB26F906B2E2CF47
:100790004F7B06B3206400C0DACF012650291570C4
:1007A00006B269F14E7F2160012F16B328C00026E2
:1007B00050294D7F06B22260102F29C001265029F2
:1007C0004B7F06B22460012F2DC016B3012650299D
:1007D000477F2860000006B22EC04F7E06B320611E
:1007E00030C0422706B3499300265029102706B28D
:1007F0004FEF10FB20F9297F16B379F2157059F1EC
:100800000126502906B2012700FB21F9237F06B3F8
:1008100071F2002650293150D0F006B2102710FB9B
:1008200022F9277E16B351F201265029012700FB39
:1008300006B223F92F7C49F2000006B3102710FB03
:1008400024F90026502906B22F7939F270CF10E42E
:100850001ABF002719C03B503195C31BD04010E48C
:100860001ABF0881033C09F10B34F9F0209189008B
:100870001981110F1213EDCF4A81441F093651F12E
:100880000D3211F0013E29F7009390003F915F91E6
:100890004F911F910F912F91DF910F90CAB7C6FD15
:1008A0001CCFCF91CFBFCF9118950091900000231E
:1008B00069F310918E00112379F534307AF1309379
:1008C0008E0000938A0010918B003BE0311B309327
:1008D0008B0024C000918E000130F4F40AE54F70C3
:1008E00049F43091610034FD1AC000936100C3E700
:1008F000D0E019C03091620034FD11C00093620055
:10090000CEE7D0E010C0052710E000C021C00527C9
:1009100010E0C89508BB14C03AE501C032ED032EC3
:10092000C0E0D0E032E017B31560C09A08B317BB3F
:1009300055E020E84FEF20FF052708BB27951795C6
:100940001C3F28F700004552B0F720FF05272795E8
:1009500008BB17951C3FB8F629913A9561F70A7FB5
:1009600010918F00110F08BBC250D04011F01093AE
:10097000890010E41ABF016017B31A7F402F4A7F25
:1009800054E05A95F1F708BB17BB48BB7FCFA0E0F6
:10099000B0E0ECECF4E0C9C0EC01688179818A81B7
:1009A0009B81611571058105910549F484E2A82EAA
:1009B00089EDB82E8BE5C82E87E0D82E02C05B01EA
:1009C0006C01C601B5012DE133EF41E050E03BD0B1
:1009D00027EA31E440E050E087D07B018C01C6017A
:1009E000B5012DE133EF41E050E02DD0CA01B9014E
:1009F00024E13BE040E050E077D0E61AF70A080B2C
:100A0000190BD801C70117FF04C081509040A040C6
:100A1000B04888839983AA83BB839F77EAE0CDB7E8
:100A2000DEB79FC0B4DF089583E690E0B0DF08959D
:100A3000A0E0B0E08093630090936400A093650011
:100A4000B0936600089597FB092E05260ED057FD3A
:100A500004D014D00AD0001C38F45095409530953D
:100A600021953F4F4F4F5F4F0895F6F79095809532
:100A7000709561957F4F8F4F9F4F0895A1E21A2E79
:100A8000AA1BBB1BFD010DC0AA1FBB1FEE1FFF1F32
:100A9000A217B307E407F50720F0A21BB30BE40B82
:100AA000F50B661F771F881F991F1A9469F76095C9
:100AB0007095809590959B01AC01BD01CF01089583
:100AC000E199FECFBFBBAEBBE09A11960DB208957F
:100AD000E199FECFBFBBAEBB0DBA11960FB6F8942D
:100AE000E29AE19A0FBE0895FF27EE27BB27AA27B7
:100AF00060FF04C0A20FB31FE41FF51F220F331FB6
:100B0000441F551F969587957795679589F70097A8
:100B1000760771F7CF01BD0108952F923F924F9252
:100B20005F926F927F928F929F92AF92BF92CF927D
:100B3000DF92EF92FF920F931F93CF93DF93CDB786
:100B4000DEB7CA1BDB0B0FB6F894DEBF0FBECDBFFE
:100B500009942A88398848885F846E847D848C84CF
:100B60009B84AA84B984C884DF80EE80FD800C81D8
:100B70001B81AA81B981CE0FD11D0FB6F894DEBFBB
:0A0B80000FBECDBFED010895FFCFB9
:080B8A00FF5A5A0100000000AF
:00000001FF
